:100000000C942B020C9448020C9448020C94480265
:100010000C9448020C9448020C9448020C94480238
:100020000C9448020C9448020C9448020C94480228
:100030000C9448020C9448020C9448020C94480218
:100040000C9448020C9448020C9448020C94480208
:100050000C944802804000000000000000000000F6
:100060000000000000000000000000000000000090
:100070000080000000000000000000000000000000
:100080000000000000000000000000000000000070
:100090000000000000000000000000000000000060
:1000A0000000000000000000000000000000000050
:1000B0000000000000000000000080800000000040
:1000C0000000000000000000000000000000000030
:1000D0000000000000000000000000000000000020
:1000E0000000000000000000008040201008040212
:1000F0000100071CE080000000000000000000007C
:1001000000000000000000000000000000000000EF
:1001100000000000000000000000000000000000DF
:1001200000000000000000000000000000000000CF
:1001300000000000804020101C060301010618602A
:10014000800000000000000000000000000000002F
:10015000000000000000000000000000000000009F
:100160000000000000000C02010000000000000080
:100170000000000000030C10000000000000000060
:10018000000000000000000000000000000000006F
:10019000000000000000000000000000000000005F
:1001A000000000000000000000000000000000400F
:1001B0002018040201000000000000000000000000
:1001C00003061C30000000000000000000000000DA
:1001D000000000000000000000000000000000001F
:1001E000000000000000000000000000000000000F
:1001F00000000000000000004040404040404040FF
:1002000040404040404040404040404040404040EE
:1002100040404040404040404040404040404040DE
:100220004040404040C0C04040404040C04040404E
:1002300040404000000000000000000000000000FE
:1002400000000000000000000000000000000000AE
:10025000000000000000000000000000000000009E
:10026000000000000000000000000000000000008E
:10027000000000000000000000000000000000007E
:10028000000000000000000000000000000000006E
:10029000000000000000000000000000000000005E
:1002A0000000000000000306080406010000000032
:1002B000000000000000000000000000000000003E
:1002C000000000000000000000000000000000002E
:1002D000000000000000000000000000000000001E
:1002E000000000000000000000000000000000000E
:1002F00000000000000000000000000000000000FE
:1003000000000000000000000000000000000000ED
:1003100000000000000000000000000000000000DD
:1003200000000000000000000000000000000000CD
:1003300000000000000000000000000000000000BD
:1003400000000000000000000000000000000000AD
:10035000000000000000000000000000000000009D
:1003600000000000000060E080E0E080E0600060ED
:10037000E080E0E080E0600060E080E0E080E0605D
:100380000000000020F8FC2404E0E0202000ECEC59
:1003900000C0E02020E0E000C0E02020E0C000FC41
:1003A000FC00ECEC20F8F820200000000000E0E069
:1003B0002020E0C000C0E0A0A0E0C020F8F820208D
:1003C000000000000000000000000000000000002D
:1003D000000000000000000000000000000000001D
:1003E0000000000000000003030000030300000001
:1003F00003030000030300000003030000030300E5
:1004000000030300000303000003030000000303D4
:1004100000010B0A0A0F0700010302020301000397
:1004200003000303000303020200030300000303AD
:1004300000000303000103020202020003030202A0
:1004400000000000000000000000000000000000AC
:1004500000000000000011241FBECFE5D8E0DEBF81
:10046000CDBF10E0A6E6B0E001C01D92A738B107ED
:10047000E1F710E0A0E6B0E0E0E3F4E102C00590AF
:100480000D92A636B107D9F70E9438080C94160AC7
:100490000C940000CF93DF93DC018038910508F0C5
:1004A00041C06034710508F03DC0CB0133E0969542
:1004B00087953A95E1F7C82FD0E0CE019695982F11
:1004C0008827979587958A0F9B1FE0916700F09189
:1004D0006800E80FF91F40816770842F90E0062EB6
:1004E00002C0959587950A94E2F780FD1BC021E034
:1004F00030E0C90102C0880F991F6A95E2F7482BC6
:100500004083E0916900F0916A00EA0FFB1F02C08E
:10051000220F331FCA95E2F78081822B808381E00E
:1005200080936600DF91CF9108951F9310916D0025
:100530000DC0812F90E06EE370E00E944A02812F8F
:1005400090E06FE370E00E944A021F5F80916D00AF
:1005500090E00F96212F30E08217930754F71F91F8
:1005600008953F924F925F926F927F928F929F92E7
:10057000AF92BF92CF92DF92EF92FF920F931F93B1
:10058000CF93DF93AA242A2D30E02F7030708A2D6C
:1005900082958F70682FF901E059FF4F808190E0BC
:1005A000062E02C0959587950A94E2F780FF5AC0FF
:1005B000C90173E0880F991F7A95E1F7362E330C45
:1005C000330CB82E282F30E0C901EC01EE24FF24B3
:1005D0004B2C5524032D10E063E0662E712C600E29
:1005E000711E52E0852E912C800E911E6801089498
:1005F000C11CD11CCE01632D70E00E944A02CE01C5
:10060000B3010E944A02E0FE03C0CE01B60102C05F
:10061000CE01B4010E944A020894E11CF11C21960B
:1006200088E0E816F10431F768010894C11CD11C78
:100630008B2D90E0B6010E944A0242E0E42EF12C9C
:10064000E00EF11E8B2D90E0B7010E944A0282015C
:10065000095F1F4FC801B6010E944A02C801B701D5
:100660000E944A02A39480E8A81609F08CCFDF917B
:10067000CF911F910F91FF90EF90DF90CF90BF909F
:10068000AF909F908F907F906F905F904F903F9032
:100690000895CF93DF93DC018038910508F044C0C2
:1006A0006034710508F040C0CB01F3E09695879562
:1006B000FA95E1F7C82FD0E0CE019695982F8827BC
:1006C000979587958A0F9B1FE0916700F0916800CE
:1006D000E80FF91F40816770842F90E08095909516
:1006E000062E02C0959587950A94E2F780FD1CC0FE
:1006F00021E030E0C90102C0880F991F6A95E2F736
:10070000809548234083E0916900F0916A00EA0FE8
:10071000FB1F02C0220F331FCA95E2F78081822B94
:10072000808381E080936600DF91CF9108952F92BE
:100730003F924F925F926F927F928F929F92AF9271
:10074000BF92CF92DF92EF92FF920F931F93DF93AE
:10075000CF9300D000D0CDB7DEB78C0169837A8308
:100760003A01FC0154900F5F1F4FF8014490015073
:100770001040CC24A1E02A2E312C1EC0EB81FC813C
:10078000849190E088219921892B29F0C701B50136
:100790000E944A0204C0C701B5010E944903D394D4
:1007A0000894E11CF11C2B813C812F5F3F4F3C835F
:1007B0002B83D51418F3C394C41400F54C2D50E0CA
:1007C000CA0187709070410102C0880C991C8A95FB
:1007D000E2F78C2D869586958695859DF0011124EE
:1007E0003296E00FF11FFC83EB8329813A81C90126
:1007F0007C01DD245A01A60CB71CDBCF0F900F90B3
:100800000F900F90CF91DF911F910F91FF90EF907C
:10081000DF90CF90BF90AF909F908F907F906F9020
:100820005F904F903F902F9008951F9310916D000F
:100830000DC0812F90E06EE370E00E944903812F8C
:1008400090E06FE370E00E9449031F5F80916D00AC
:1008500090E00F96212F30E08217930754F71F91F5
:100860000895AC9AAC9800000000000000000895C4
:100870008BBB80E090E001C00000019684319105BF
:10088000D9F7AC9AAC980000000000000000089571
:10089000AD988BBB80E090E001C0000001968431F0
:1008A0009105D9F7AC9AAC98000000000000000058
:1008B000AD9A089581708E630E94480408958F73E5
:1008C00080640E94480408958770886B0E944804E1
:1008D0000895DF92EF92FF920F931F93CF93DF93D0
:1008E00080916600882309F4A8C010926600AF9A30
:1008F000AE98C0E0D0E0DC2EE0916900F0916A0093
:10090000EC0FFD1F8081882309F43FC07E0100E0C9
:1009100010E0E0916900F0916A00EC0FFD1F80810A
:1009200090E0002E02C0959587950A94E2F780FF2B
:100930001CC08D2D0E945F04802F0E946404E091F2
:100940006700F0916800EE0DFF1D80818BBB80E099
:1009500090E001C00000019684319105D9F7AC9A6E
:10096000AC9800000000000000000F5F1F4F80E8FF
:1009700090E0E80EF91E0830110559F6E091690083
:10098000F0916A00EC0FFD1F10822196C034D10552
:1009900009F0B1CFAE9AAF98B0E4DB2E0D2D10E088
:1009A000E0916900F0916A00E00FF11F80818823D7
:1009B00009F43EC07801C0E0D0E0E0916900F09118
:1009C0006A00E00FF11F808190E00C2E02C0959527
:1009D00087950A94E2F780FF1CC08D2D0E945F046A
:1009E0008C2F0E946404E0916700F0916800EE0D86
:1009F000FF1D80818BBB80E090E001C0000001966C
:100A000084319105D9F7AC9AAC9800000000000041
:100A10000000219680E890E0E80EF91EC830D1056C
:100A200061F6E0916900F0916A00E00FF11F108219
:100A3000D39490E8D91609F0B1CFDF91CF911F91EF
:100A40000F91FF90EF90DF90089524EF31E040E0A8
:100A500050E00E94D00901C0000061507040804009
:100A60009040D1F7089501C000006150704080406F
:100A70009040D1F708951F93AE9AAF9A80E00E94FC
:100A80005F0410E0812F0E94640420E030E01BBA74
:100A900080E090E001C00000019684319105D9F713
:100AA000AC9AAC9800000000000000002F5F3F4FA0
:100AB0002034310561F71F5F183021F780E00E9474
:100AC0005F0480E00E946404E0916700F091680098
:100AD00080E094E0DF019C011D9221503040E1F75D
:100AE000E0916900F0916A0080E8DF011D928A952B
:100AF000E9F71F910895AE9AAF9A81E00E945A04D7
:100B000080EC0E9448040E943B0508950E943B052A
:100B100088E380936D0080E4809382008CE380936F
:100B2000800081E090E090936C0080936B008FEFE9
:100B30009FEF90936F0080936E001092810080E78A
:100B400090E06FEF70E040E150E00E94C9090E9420
:100B500095020E94B10208954F925F926F927F9228
:100B60008F929F92AF92BF92CF92DF92EF92FF92BD
:100B70000F931F93CF93DF938091820090E0609159
:100B8000800070E06150704001970E9449036091BD
:100B9000800070E0615070408091820090E00E947F
:100BA00049038091820090E06091800070E0615084
:100BB000704001960E9449038091820090E060910C
:100BC0008000019770E00E9449036091800080914D
:100BD000820090E070E00E9449038091820090E0E2
:100BE00060918000019670E00E944903809182002C
:100BF00090E06091800070E06F5F7F4F01970E94EE
:100C000049036091800070E06F5F7F4F80918200A8
:100C100090E00E9449038091820090E06091800002
:100C200070E06F5F7F4F01960E94490380918100C1
:100C3000882309F4AAC120916B0030916C00809147
:100C40008200820F8093820060916E0070916F002D
:100C500040918000460F40938000823010F481E084
:100C600003C08E3758F08EE780938200882799273B
:100C7000821B930B90936C0080936B00423090F436
:100C800081E08093800088279927861B970B90939B
:100C90006F0080936E0099247724662441E0442EEF
:100CA000512C3CC04C33A9F480918200482F50E075
:100CB00080916D00282F30E0CA01019682179307BA
:100CC00054F341505040205F3F4F241735071CF329
:100CD000DACF4F3301F780916D00885F80938200F7
:100CE0008CE38093800081E090E090936C0080938F
:100CF0006B008FEF9FEF90936F0080936E001092C8
:100D000081000E94950280E291EAA7E0B0E001C074
:100D100000000197A109B109D9F7BDCFA92DB0E015
:100D2000AF70B070FD01E059FF4FB080892D829502
:100D30008F70F82E8B2D90E00F2C02C09595879523
:100D40000A94E2F780FFA1C0EA2EEE0CEE0CEE0C46
:100D50008091820090E06C010894C11CD11C2E2D62
:100D600030E0C216D3060CF490C0FC013197E901C3
:100D70002796CE17DF070CF488C08F2C880C880CC0
:100D80008091800090E0AC014F5F5F4F682D70E074
:100D9000461757070CF479C001978B010D5F1F4F61
:100DA000081719070CF471C04617570719F0801778
:100DB000910799F5A059BF4FC20102C0880F991F32
:100DC000FA94E2F780958B218C93CE2DD0E05B01D5
:100DD0000894A11CB11C32E0E32EF12CE60EF71EA4
:100DE00028E0C22ED12CCC0EDD1ECE01682D70E085
:100DF0000E944903CE01B5010E944903CE01B7010B
:100E00000E944903CE01B8010E9449032196CC15E6
:100E1000DD0559F76624639438C0C216D30619F06D
:100E2000EC17FD0791F5A059BF4FC20102C0880F12
:100E3000991FFA94E2F780958B218C93CE2DD0E008
:100E40005B010894A11CB11C92E0E92EF12CE60E86
:100E5000F71E88E0C82ED12CCC0EDD1ECE01682DE9
:100E600070E00E944903CE01B5010E944903CE0102
:100E7000B7010E944903CE01B8010E94490321969F
:100E8000CC15DD0559F777247394939480E8981670
:100E900009F044CF772091F080916B0090916C0025
:100EA000909581959F4F90936C0080936B00880F75
:100EB000991F20918200280F20938200662091F0D4
:100EC00080916E0090916F00909581959F4F9093C7
:100ED0006F0080936E00880F991F20918000280F6B
:100EE00020938000772019F4662009F456C0809181
:100EF0007000882309F051C080917200882309F0A6
:100F00004CC080917300882309F047C08091740021
:100F1000882309F042C080917500882309F03DC004
:100F2000809176008823C9F5809177008823A9F500
:100F300080917800882389F580917900882369F56C
:100F400080917A00882349F580917B00882329F5D8
:100F500080917C00882309F580917D008823E9F445
:100F600080917E008823C9F480917F008823A9F4B2
:100F700080E291EAA7E0B0E001C000000197A1097A
:100F8000B109D9F70E94860508C080916D00885F7D
:100F9000809382008CE3809380008091820090E0B7
:100FA0006091800070E06150704001970E944A0299
:100FB0006091800070E0615070408091820090E00C
:100FC0000E944A028091820090E06091800070E06F
:100FD0006150704001960E944A028091820090E028
:100FE00060918000019770E00E944A026091800049
:100FF0008091820090E070E00E944A02809182001D
:1010000090E060918000019670E00E944A02809119
:10101000820090E06091800070E06F5F7F4F0197E9
:101020000E944A026091800070E06F5F7F4F809164
:10103000820090E00E944A028091820090E06091DC
:10104000800070E06F5F7F4F01960E944A02DF913F
:10105000CF911F910F91FF90EF90DF90CF90BF90B5
:10106000AF909F908F907F906F905F904F9008957A
:101070001F93CF93DF938FEF8ABB88EF84BB1BBA9C
:1010800015BAAB9A80E094E00E94C4088093670090
:101090009093680080E890E00E94C4088093690003
:1010A00090936A00AC9880E090E001C00000019647
:1010B00023EC80359207D1F70E947B05AB9884E53D
:1010C00090E060E070E040E050E00E9497030E94F2
:1010D0006904989BFECF80E090E001C0000001967B
:1010E00023E188389207D1F79899FECF80E090E00D
:1010F00001C00000019623E188389207D1F70E94D1
:101100008605C0E0D0E011E09A9B0DC080916D0093
:10111000882349F00E94150480916D0081508093CE
:101120006D000E949502999B0DC080916D008037E3
:1011300048F40E94150480916D008F5F80936D00CC
:101140000E94950280918100882321F4989B02C01F
:10115000109381002196CE0163E070E00E94EF09B8
:10116000892B21F080918100882311F40E94AC0525
:1011700080E090E001C0000001962AE388399207E0
:10118000D1F70E946904C0CFCF93DF93BC018230B6
:10119000910510F462E070E0A0918500B0918600A6
:1011A000ED01E0E0F0E040E050E021C0888199816D
:1011B0008617970769F48A819B81309719F093838A
:1011C000828304C09093860080938500FE0134C022
:1011D0006817790738F44115510519F084179507F8
:1011E00008F4AC01FE018A819B819C01E9012097F2
:1011F000E9F641155105A9F1CA01861B970B049721
:1012000008F4BA01E0E0F0E02AC08D919C911197BA
:1012100084179507F9F46417750781F412968D9178
:101220009C911397309719F09383828304C0909315
:10123000860080938500FD0132964FC0CA01861B4F
:10124000970BFD01E80FF91F6193719302978D933E
:101250009C9343C0FD01828193819C01D901109729
:10126000A1F68091830090918400892B41F48091B4
:10127000620090916300909384008093830040917A
:101280006400509165004115510541F44DB75EB7BA
:101290008091600090916100481B590B2091830060
:1012A0003091840024173507B0F4CA01821B930BD8
:1012B0008617970780F0AB014E5F5F4F8417950745
:1012C00050F0420F531F5093840040938300F90164
:1012D0006193719302C0E0E0F0E0CF01DF91CF9124
:1012E0000895CF93DF93009709F450C0EC01229743
:1012F0001B821A82A0918500B0918600109709F197
:1013000040E050E0AC17BD0708F1BB83AA83FE01A3
:1013100021913191E20FF31FAE17BF0779F48D9140
:101320009C911197280F391F2E5F3F4F39832883D7
:1013300012968D919C9113979B838A834115510539
:1013400071F4D0938600C093850020C012968D91D1
:101350009C911397AD01009711F0DC01D3CFFA01F6
:10136000D383C28321913191E20FF31FCE17DF07A0
:1013700069F488819981280F391F2E5F3F4FFA0148
:10138000318320838A819B8193838283DF91CF91F4
:101390000895DC0101C06D9341505040E0F708957D
:1013A000629FD001739FF001829FE00DF11D649F49
:1013B000E00DF11D929FF00D839FF00D749FF00DD5
:1013C000659FF00D9927729FB00DE11DF91F639F76
:1013D000B00DE11DF91FBD01CF011124089597FB48
:1013E000092E07260AD077FD04D00CD006D00020A5
:1013F0001AF4709561957F4F0895F6F79095819551
:101400009F4F0895AA1BBB1B51E107C0AA1FBB1F1A
:10141000A617B70710F0A61BB70B881F991F5A9580
:10142000A9F780959095BC01CD010895F894FFCF60
:061430002000870000000F
:00000001FF
